:1000000012C02AC029C028C027C026C0ACC124C045
:1000100023C022C021C020C01FC01EC01DC01CC0E4
:100020001BC01AC019C011241FBECFEDCDBF10E0F8
:10003000A0E6B0E0EAEDF4E002C005900D92A8362B
:10004000B107D9F710E0A8E6B0E001C01D92AC38C6
:10005000B107E1F7B2D03FC2D3CF80B38095382F3C
:100060008091660032FF14C0882309F44FC081508C
:1000700080936600882309F049C090E08091860053
:10008000882309F491E090938600109287003EC087
:100090008B3F08F038C080918600882371F0209152
:1000A0008A002F3180F52F5F20938A002150E1993B
:1000B000FECF1CBA81E090E01FC0809187008823AA
:1000C00071F080918B008830F0F4282F2F5F2093FF
:1000D0008B00E199FECF1CBA82E090E00DC08091C8
:1000E00089008B3080F0282F245020938900E199DB
:1000F000FECF1CBA80E090E08EBB2DBB0FB6F8940B
:10010000E29AE19A0FBE8FEF8093660080916500BE
:1001100033FF14C0882309F44FC0815080936500D9
:10012000882309F049C090E080918700882309F472
:1001300091E0909387001092860008958B3F08F01D
:1001400038C080918600882371F020918A00233086
:1001500080F1215020938A002F5FE199FECF1CBAD5
:1001600081E090E01FC080918700882371F080912A
:100170008B008823F1F0282F215020938B00E199E8
:10018000FECF1CBA82E090E00DC080918900893CCE
:1001900080F4282F2C5F20938900E199FECF1CBAB0
:1001A00080E090E08EBB2DBB0FB6F894E29AE19A06
:1001B0000FBE8FEF809365000895CF92DF92EF928C
:1001C000FF920F931F93CF93DF938FEF87BB8CE04A
:1001D00082BB81E790E0909382008093810089E761
:1001E00090E0909384008093830089B7826089BFF8
:1001F00081E083BF7894E199FECF80E090E08EBBF0
:10020000E09A8DB3809389008F3F19F487E3809340
:100210008900E199FECF81E090E08EBBE09A8DB33A
:1002200080938A008F3F19F486E080938A00E199D9
:10023000FECF82E090E08EBBE09A8DB380938B007E
:100240008F3F19F482E080938B00D090640000917E
:10025000700010916300E0908800F0906200CC2460
:10026000C394C0EDD7E0FA9489F4F0908A00E8E6F0
:10027000F0E0808190E06CED70E0F4D0892F990F70
:10028000990B819380E0E037F80799F74091890056
:10029000083088F4242F30E0E02FFF27E7FDF095A9
:1002A000E859FF4FC901811B91096FEF70E0DAD067
:1002B000B901EAD06083115011F580918B00DD20E7
:1002C00069F00F5F90E00696202F332727FD3095C9
:1002D000821793079CF4142FDD2411C00150202FA6
:1002E000332727FD309590E0909581959F4F821799
:1002F000930724F0142FDD24D39401C0142F809190
:100300008600882311F0E7FE06C0809187008823CD
:1003100081F0E4FC0EC080E090E0E0918300F09179
:100320008400E80FF91F1082019688309105A9F723
:1003300012C020E030E0E0918300F0918400E20FF1
:10034000F31FD901A859BF4F8C9180832F5F3F4F76
:100350002830310581F7C09285007FDECE010197FC
:10036000F1F7E39480CF1F920F920FB60F921124F2
:100370002F933F934F938F939F93EF93FF9380918E
:10038000610088BB409160004F5F40936000442350
:10039000C9F480918500882391F010928500209106
:1003A000830030918400809181009091820090932D
:1003B00084008093830030938200209381008FEF2C
:1003C00080936100E0918100F09182008081841728
:1003D00029F4809161008E7F809361008181841770
:1003E00029F4809161008D7F809361008281841760
:1003F00029F4809161008B7F809361008381841751
:1004000029F480916100877F809361008481841743
:1004100029F4809161008F7E80936100858184172B
:1004200029F4809161008F7D80936100868184171B
:1004300029F4809161008F7B80936100878184170C
:1004400029F4809161008F7780936100FF91EF9193
:100450009F918F914F913F912F910F900FBE0F90D1
:100460001F9018955527002480FF02C0060E571FC5
:10047000660F771F6115710521F096958795009796
:1004800099F7952F802D089597FB092E07260AD0FE
:1004900077FD04D00CD006D000201AF47095619539
:1004A0007F4F0895F6F7909581959F4F0895AA1B69
:1004B000BB1B51E107C0AA1FBB1FA617B70710F04F
:1004C000A61BB70B881F991F5A95A9F78095909581
:0A04D000BC01CD010895F894FFCFA0
:0804DA00FFFF010101FFFF001B
:00000001FF
